:100EA400EA600001010100000201010301010401E3
:100EB4000105010106010107010108010109010100
:100EC4000A01010B00000C00000D00000E00000FD1
:100ED40000001000001100001200001300001400B4
:100EE400001500001600001700001800001900008B
:030EF400FAFAFA0D
:10004800750B00750A00AE0AAF0BAC08AD09EDC31D
:100058009FEC9E401674FF12002E75CF01780B742A
:100068000126F6500418E436F650DB22C2AF75D9E3
:1000780004758F0375B7A575B7F190F800E4F075AE
:100088008F0175B7A575B7F1740690F800F075B7CC
:10009800A575B7F190F801E4F075B7A575B7F190BB
:1000A8000036E090F802F075B7A575B7F190003A00
:1000B800E090F803F075B7A575B7F1900037E090B8
:1000C800F804F075B7A575B7F1900038E090F80519
:1000D800F075B7A575B7F1900039E090F806F0759E
:1000E800B7A575B7F190003BE090F807F0758F0061
:1000F800900014E0900017F0900015E0900018F0C0
:10010800900016E0900019F075D944D2AF22900003
:100118005AE0B4AB61C2AF75D90475B62275F52241
:10012800758F0375B7A575B7F1740090F600F07573
:100138008F01752C00752B00AE2BAF2C7413BE00ED
:10014800279F402475B7A575B7F1900022120EF7C6
:10015800E0FC90F600120EF7ECF0782C740126F60D
:10016800500418E436F650D0758F0075F51175B641
:100178002075D944D2AF2290005AE0B4AA02800375
:100188000202BCC2AF75D90475B62275F522758F07
:100198000375B7A575B7F1740090EE00F075B7A5B3
:1001A80075B7F1740090F000F075B7A575B7F174E4
:1001B8000090F200F075B7A575B7F1740090F400DF
:1001C800F0758F01752C00752B00AE2BAF2C74FFCA
:1001D800C39F74019E402475B7A575B7F190005B65
:1001E800120EF7E0FC90EE00120EF7ECF0782C748B
:1001F8000126F6500418E436F650CF752C00752BFE
:1002080000AE2BAF2C74FFC39F74019E402475B7BA
:10021800A575B7F190025B120EF7E0FC90F00012A2
:100228000EF7ECF0782C740126F6500418E436F634
:1002380050CF752C00752B00AE2BAF2C74FFC39FCD
:1002480074019E402475B7A575B7F190045B120E32
:10025800F7E0FC90F200120EF7ECF0782C7401260F
:10026800F6500418E436F650CF752C00752B00AE06
:100278002BAF2C74FFC39F74019E402475B7A575DE
:10028800B7F190065B120EF7E0FC90F400120EF73F
:10029800ECF0782C740126F6500418E436F650CFAA
:1002A800758F0075F51175B62075D944D2AF743ABB
:1002B80090075BF02290005AE0B4AA028003020380
:1002C800FAC2AF75D90475B62275F522758F037514
:1002D800B7A575B7F1740090E600F075B7A575B7C6
:1002E800F1740090E800F075B7A575B7F174009047
:1002F800EA00F075B7A575B7F1740090EC00F075D9
:100308008F01752C00752B00AE2BAF2C74FFC39F8B
:1003180074019E402475B7A575B7F190005B120E65
:10032800F7E0FC90E600120EF7ECF0782C7401264A
:10033800F6500418E436F650CF752C00752B00AE35
:100348002BAF2C74FFC39F74019E402475B7A5750D
:10035800B7F190025B120EF7E0FC90E800120EF77E
:10036800ECF0782C740126F6500418E436F650CFD9
:10037800752C00752B00AE2BAF2C74FFC39F740136
:100388009E402475B7A575B7F190045B120EF7E08F
:10039800FC90EA00120EF7ECF0782C740126F65067
:1003A8000418E436F650CF752C00752B00AE2BAF31
:1003B8002C74FFC39F74019E402475B7A575B7F1CF
:1003C80090065B120EF7E0FC90EC00120EF7ECF0D2
:1003D800782C740126F6500418E436F650CF758F41
:1003E8000075F51175B62075D944D2AF743A9007E7
:1003F8005BF022C2AF75D90475F522752C00752BF8
:1004080000AE2BAF2C74FFC39F74019E401F90EE6B
:1004180000120EF7E493FC90005B120EF7ECF078F4
:100428002C740126F6500418E436F650D4752C00C6
:10043800752B00AE2BAF2C74FFC39F74019E401F19
:1004480090F000120EF7E493FC90025B120EF7ECAA
:10045800F0782C740126F6500418E436F650D4755A
:100468002C00752B00AE2BAF2C74FFC39F74019E1C
:10047800401F90F200120EF7E493FC90045B120EFA
:10048800F7ECF0782C740126F6500418E436F65090
:10049800D4752C00752B00AE2BAF2C74FFC39F7442
:1004A800019E401F90F400120EF7E493FC90065B47
:1004B800120EF7ECF0782C740126F6500418E43686
:1004C800F650D475F51175D944D2AF743A90075BDC
:1004D800F022752E00752D0075F809AE2DAF2E741B
:1004E80027BE0004D39F50030205B0A2F9B35003FE
:1004F8000205ADE52E452D700375A3D2AE2DAF2EA6
:1005080074016F4E700375A300AE2DAF2E74026F89
:100518004E700BE52A75F002A4FDACF08DA3AE2D4C
:10052800AF2E74036F4E700375A300AE2DAF2E74FB
:10053800046F4E700375A300AE2DAF2E74056F4E79
:10054800700375A300AE2DAF2E74066F4E70037541
:10055800A300AE2DAF2E74076F4E700375A300AEC7
:100568002DAF2E74086F4E700375A300AE2DAF2EFD
:100578007408BE00039F500C900033120EF7E5A3D9
:10058800F075A300AE2DAF2E74266F4E700574144F
:1005980012002EAE2DAF2E74266F4E700375F80D17
:1005A800782D120F150204E32290005AE0B4AB0232
:1005B8008003020649752E00752D0075F809AE2DC9
:1005C800AF2E7427BE007AD39F4076A2F9B3406E4F
:1005D800E52E452D700375A382AE2DAF2E74016FE5
:1005E8004E700375A300AE2DAF2E74026F4E700BC4
:1005F800E52A75F002A4FDACF08DA3AE2DAF2E74E4
:10060800036F4E700375A300AE2DAF2E7403BE00AA
:10061800039F5009900038120EF7E0F5A3AE2DAFF6
:100628002E74266F4E7005741412002EAE2DAF2E48
:1006380074266F4E700375F80D782D120F1502058C
:10064800C622900004E0FEA3E0FF900EA6120EF76B
:10065800E493F59974506F4E7003752F0090000461
:1006680012001E22C203C20422C293C294C291C2C3
:1006780092C287C290E5B554EFF5B5E5B554DFF5FC
:10068800B5C296C295C2A0C297C2A2C2A1E5B5548E
:10069800BFF5B5E5B5547FF5B5E5B554FBF5B5221D
:1006A800E53064046006E59964FF6002802DA200CD
:1006B8004004D2008023E530600674E62530F53F1B
:1006C800E52F600674F0252FF53FE530B401028070
:1006D800FE753000752F00C2008002C200E5309020
:1006E8000E32F8282873753000E599B4FF03752F8A
:1006F80001E599B4FE03752F02E599B4FD03752F42
:1007080003E599B4FC03752F04E599B4FA03752F32
:1007180005E599B4FB06753001120671E599B4F93F
:1007280006753004120671900004E4F0A3F0D29923
:100738000209DE900004E0FEA3E0FF90005B120EC9
:10074800F7E599F090000412001E900004E0FEA363
:10075800E0FFEFB40106EEB407028003020802903E
:10076800075BE0B43C0280030207F975FFA0C29C56
:1007780012066C9000F9E0900022F0900068E0907A
:100788000023F0900088E0900024F09000B1E09001
:100798000025F090005DE0900026F09000A3E09026
:1007A8000027F09000C1E0900028F0900095E090BC
:1007B8000029F09000B3E090002AF09000E3E09068
:1007C800002BF0740090002CF0740090002DF07451
:1007D8000090002EF074AB90005AF012011674AA23
:1007E80090005AF012017F1202BDD29C7599FB80CD
:1007F800FE7599FF753000752F000209DE0209DECB
:100808000209DE900004E0FEA3E0FF90005B120EF8
:10081800F7E599F090000412001E900004E0FEA392
:10082800E0FFEFB40006EEB4010280030209DE75B2
:10083800FFA0900016E0D394C7400B900016E0C3C9
:1008480094C8F532801A900016E0D39463400B9058
:100858000016E0C39464F5328006900016E0F53285
:10086800E53275F002A4FFAEF08F44EF90005B1202
:10087800003EEFFCE0FDEC90005E12003EEDFCE077
:10088800FDEC2DB5320280030209D00FEF90005B1A
:1008980012003EE544FFE0FCEF90005F12003EECE2
:1008A800FFE0FCEFC39CB5320280030209D0E544A7
:1008B80090005D12003EE544FFE0FCEF90006012FE
:1008C800003EECFFE0FCEF2CB5320280030209D0B9
:1008D800E54490006112003EE0C39532900036F086
:1008E800E54490006212003EE0C39532900037F074
:1008F800E54490006512003EE0C39532900038F060
:10090800E54490006612003EE0C39532900039F04D
:10091800E54490006712003EE0C3953290003AF03B
:10092800E54490006812003EE0C3953290003BF029
:1009380012007474FF90003CF074FF90003DF07456
:10094800FF90003EF074FF90003FF074FF9000406D
:10095800F074FF900041F074FF900042F074FF9033
:100968000043F074AB90005AF0752A6475290012A0
:1009780005B1750964750800120048752A6575295E
:10098800001205B1750964750800120048752A66D9
:100998007529001205B175096475080012004875BB
:1009A8002A677529001205B17509647508001200D7
:1009B80048752A687529001205B17509647508001B
:1009C8001200487599F980FE7599FF7509647508D4
:0609D8000012004880FE41
:0F0E32000206EE02073B02080502080802080B41
:1009DE0022E52F900E41F8282873020AE0900004B9
:1009EE00E0FEA3E0FF900006120EF7E0F5999000EE
:1009FE000412001E900004E0FEA3E0FF741C6F4E74
:100A0E007003752F00020AE0854199020AE09000FA
:100A1E0004E0FEA3E0FF90005B120EF7E0F599EF05
:100A2E00B40107EEB40703752F0090000412001EE8
:070A3E00020AE0900005E050
:0F0E41000209E80209EB020A16020A1C020A4122
:100A4500900E53F8282873852699020AD5759900C2
:100A5500807E85339980798534998074853899802D
:100A65006F853A99806A853B998065853C99806058
:100A7500853D99805B853E9980568539998051756C
:100A85009900804C75990080477599008042853F93
:100A950099803D7599008038759900803375990066
:100AA500802E75990080297599008024759900809C
:100AB5001F759900801A7599008015759900801029
:100AC500759900800B75990080067599FC752F0046
:100E5300020A4C020A52020A57020A5C020A61029F
:100E63000A66020A6B020A70020A75020A7A020A09
:100E73007F020A84020A89020A8E020A93020A98EE
:100E8300020A9D020AA2020AA7020AAC020AB102DE
:100E93000AB6020ABB020AC0020AC5020ACA020A49
:010EA300CF7F
:0B0AD50090000412001E800312064A6D
:030E5000020ADDB6
:100AE00022C2CF05372290F800E493640660089094
:100AF0000047E493B40602800280FE75840175A766
:100B00000075FF8075EF0690005AE4F075C9107506
:100B1000A70F75A1C775A70075D90075CE0C75A76D
:100B20000F75F1FE75F2FF75F30775F47875A4BAC9
:100B300075A5FF75A60775AE0075AFFF75D48175F5
:100B4000D5FF75D6FF75D7FF75A70075A20175A1F2
:100B50004775F80975D80075D90475DA0975DB0988
:100B600075E60875BC0175BE0475BD6C75BE07756C
:100B7000BDA075BE0875BD0175BC0075BB1875BC00
:100B80002075BA0875E88075D11375A70F75E10552
:100B900075E20075C74075B500C293C294C291C298
:100BA00092C287C290E5B554EFF5B5E5B554DFF5CF
:100BB000B5C296C295C2A0C297C2A2C2A1E5B55461
:100BC000BFF5B5E5B5547FF5B5E5B554FBF5B5759D
:100BD0009700759780740A12002E7597C0E5975498
:100BE00020700280F8758F0275A700D2AF7598004B
:100BF00075A90C75A70F75AB4375ADFB75AC1E756C
:100C0000A700758912758E04758C00758A00C2A9BB
:100C1000D28CD2ADC2CFD2CA75B62075D944752F49
:100C200000753000C2997509C87508001200487532
:100C3000A70FE5FC900013F0E5FB900014F0E5FA37
:100C4000900015F0E5F9900016F075A7001203FB6F
:100C500090F800E493B4066E90F800E493900006D8
:100C6000F090F802E493900009F090F803E4939078
:100C7000000AF090F804E49390000BF090F805E47B
:100C800093900011F090F806E493900012F0900019
:100C900014E0900017F0900015E0900018F090001C
:100CA00016E0900019F090F807E493900020F0907F
:100CB0000020E0440A900020F0900020E054FE90D4
:100CC0000020F0020D487406900006F0900047E402
:100CD00093B40629752A647529001204DA752AC8A6
:100CE00075290090003CE0900017F090003DE090E6
:100CF0000018F090003EE0900019F08012746390AC
:100D00000017F07463900018F07463900019F07588
:100D10002A667529001204DA752AC8752900900020
:100D20003CE0900009F0900043E090000AF0900051
:100D30003DE090000BF07400900011F07401900001
:100D400012F07400900020F07400900007F0740A14
:100D5000900008F0740090000CF074F490000DF016
:100D6000740490000EF0740090000FF07405900071
:100D700010F0740090001AF0740090001BF07400E2
:100D800090001CF0740090001DF0740090001EF0A4
:100D9000740090001FF074FF900021F0C2009000DA
:100DA00004E4F0A3F07400900068F075271975282A
:100DB00064900002740DF0A374ACF0753100743AC5
:100DC00090075BF074FD90075CF0753FFA75430087
:100DD000752600752500753600753300753E007563
:100DE0003400753800753900753A00753B00753C64
:100DF00000753D00900000E4F0A3F07540007541DF
:100E000001D29CD2EC75CF01A298B34005C29812D2
:100E100006A8E52F6006A299B3B340028005C299E7
:100E20001209DFE53064016005E530B4040280D5C5
:020E300080D36D
:09003E002582F58250020583229F
:080F15000806B60002180622CE
:0D001E00A3E004F07006120F02E004F022CF
:10002E00600D782B020038007830D8FED5E0F8222B
:03002B00020003CD
:03000000020F0CE0
:090F0C0075814675D000020AE669
:100EF700E5822FF582E5833EF583220582D58202BE
:050F0700158315822294
:10000300C0E0C0F0C083C082C0D075D000120AE146
:0B001300D0D0D082D083D0F0D0E032FB
:00000001FF
